:100000000C942A000C943C000C943C000C943C0092
:100010000C943C000C943C000C943C000C943C0070
:100020000C943C000C943C000C943C000C9482001A
:100030000C943C000C943C000C943C000C943C0050
:100040000C943C000C943C000C943C000C943C0040
:100050000C943C0011241FBECFE5D4E0DEBFCDBF21
:1000600010E0A0E6B0E001C01D92A23AB107E1F7AE
:100070000E943E000C9440010C940000DF93CF934B
:1000800000D000D00F92CDB7DEB784B38FEF84BB22
:1000900080EA91E00E9473000E940B018823E1F343
:1000A0000E94DA008134C1F70E940B018823E1F33A
:1000B0000E94DA00813481F70E940B018330E1F75E
:1000C0000E94DA008B830E94DA008C830E94DA009F
:1000D000282F8D839B818C8180959817E9F62A358E
:1000E000D9F695BBD9CF2FEF209361002091610005
:1000F0002093600090BD89B986E880BD80E98AB907
:10010000789408951F920F920FB60F9211242F9397
:100110003F934F938F939F93EF93FF934CB18091B5
:1001200061008F3389F180916100209160009927EF
:1001300087FD90950196332727FD30958217930709
:1001400039F1809161008F3391F1809161008F5F6F
:1001500080936100E0916100FF27E7FDF095EE5983
:10016000FF4F4083809160008F3F11F41092600038
:10017000FF91EF919F918F914F913F912F910F9010
:100180000FBE0F901F90189580916000882359F63C
:10019000809160008F5F8093600080916000803468
:1001A00081F610926000809161008F3371F6109299
:1001B0006100D0CF809160008F3FC9F0E091600076
:1001C000FF27E7FDF095EE59FF4FE0819091600029
:1001D00080916100981771F0809160008F5F80932B
:1001E000600080916000803471F08E2F0895E0E00F
:1001F0008E2F08958FEF809361008091610080932E
:1002000060008E2F0895109260008E2F08955D9BE0
:10021000FECF8CB90895809160008F3FE1F09091FE
:10022000600080916100981774F090916000809157
:10023000610089179CF490916100809160009F5B40
:10024000981B892F089590916100809160009F5FB5
:10025000981B892F089590E0892F089591E0892FA8
:100260000895FC018081882339F05D9BFECF8CB915
:10027000319680818823C9F75D9BFECF1CB8089515
:04028000F894FFCF20
:00000001FF
